:1000000013C06AC096C034C033C032C031C030C0E3
:100010002FC058C22DC052C12BC02AC029C028C031
:1000200027C026C025C0A50511241FBECFE5D4E0FA
:10003000DEBFCDBF10E0A0E6B0E0E0EFFDE002C023
:1000400005900D92AA3FB107D9F711E0AAEFB0E0F1
:1000500001C01D92A938B107E1F710E0C8E2D0E075
:1000600003C02297FE0189D6C632D107D1F792C2CA
:10007000C7CF8230E8F4E82FFF27EE0FFF1FE650CE
:10008000FF4F71836083882341F485B78C7F842B75
:1000900085BF8BB780648BBF089585B7837F440F7E
:1000A000551F440F551F842B85BF8BB780688BBFAE
:1000B0000895E82F823078F4882319F48BB78F7B6A
:1000C00002C08BB78F778BBFFF27EE0FFF1FE65065
:1000D000FF4F1182108208951F920F920FB60F9258
:1000E00011242F933F934F935F936F937F938F933D
:1000F0009F93AF93BF93EF93FF938091FA009091FA
:10010000FB00892B29F0E091FA00F091FB000995A2
:10011000FF91EF91BF91AF919F918F917F916F91DF
:100120005F914F913F912F910F900FBE0F901F90B5
:1001300018951F920F920FB60F9211242F933F9391
:100140004F935F936F937F938F939F93AF93BF93DF
:10015000EF93FF938091FC009091FD00892B29F093
:10016000E091FC00F091FD000995FF91EF91BF91A6
:10017000AF919F918F917F916F915F914F913F913F
:100180002F910F900FBE0F901F901895880F991FF9
:10019000880F991FE0919800F0919900E80FF91FDE
:1001A000808191810895880F991F880F991FE09190
:1001B0009800F0919900E80FF91F828193810895CA
:1001C000880F991FE0917A00F0917B00E80FF91FEA
:1001D000808191810895880F991F880F991FE09160
:1001E0006000F0916100E80FF91F8281938108950A
:1001F000EF92FF920F931F937B018C0122E030E07E
:1002000040E050E089D5205C3D4B404F5F4FCA0134
:10021000B901A801970180D521503040404050409D
:10022000BB2757FDBA95A52F942F832F2F5F3F4FE4
:100230004F4F5F4F80BD215029B9549A539A579A16
:100240001F910F91FF90EF9008955D9BFECF8CB9A9
:10025000089580910001909101012091FE0030915C
:10026000FF00821B930B60E870E021D50895409158
:10027000FE005091FF0080910001909101018417D0
:10028000950719F48FEF9FEF0895FA01E75FFE4F8E
:100290002081CA01019660E870E009D59093FF00C3
:1002A0008093FE00822F992708958091FE009091FF
:1002B000FF00909301018093000108951F920F9217
:1002C0000FB60F9211242F933F934F935F936F9329
:1002D0007F938F939F93AF93BF93EF93FF934CB113
:1002E000E0910001F0910101CF01019660E870E01A
:1002F000DED49C018091FE009091FF002817390701
:1003000039F0E75FFE4F40833093010120930001F5
:10031000FF91EF91BF91AF919F918F917F916F91DD
:100320005F914F913F912F910F900FBE0F901F90B3
:10033000189508958ADF08958AE0FCDF0895CF9329
:10034000DF93EC0102C02196F5DF88818823D9F77D
:10035000DF91CF9108952F923F924F925F926F92CB
:100360007F928F929F92AF92BF92CF92DF92EF9245
:10037000FF920F931F93CF93DF93CDB7DEB7A09774
:100380000FB6F894DEBF0FBECDBF6B017C01190123
:100390002A01611571058105910519F480E3CADF11
:1003A00048C06624772443015E010894A11CB11C57
:1003B0008501060D171DC701B601A20191018AD45E
:1003C000F80160830894611C711C811C911CC70199
:1003D000B601A20191017ED469017A01211531058E
:1003E0004105510529F773010894E108F108EA0C69
:1003F000FB1CAA24BB24650110C0F70180818A3050
:1004000010F4805D01C0895C95DF0894A108B108F3
:10041000C108D1080894E108F10888279927DC0170
:1004200086199709A809B909A816B906CA06DB06EC
:1004300021F7A0960FB6F894DEBF0FBECDBFDF91B7
:10044000CF911F910F91FF90EF90DF90CF90BF90D1
:10045000AF909F908F907F906F905F904F903F9064
:100460002F900895EF92FF920F931F937B018C01C1
:1004700097FF0AC08DE25EDF10950095F094E0943E
:10048000E11CF11C011D111D2AE030E040E050E0AC
:10049000C801B70160DF1F910F91FF90EF900895A1
:1004A00020E130E040E050E056DF089528E030E001
:1004B00040E050E050DF089522E030E040E050E0BE
:1004C0004ADF08951F920F920FB60F9211248F9357
:1004D0009F93AF93BF938091050190910601A091E6
:1004E0000701B09108010196A11DB11D809305017E
:1004F00090930601A0930701B0930801BF91AF91BB
:100500009F918F910F900FBE0F901F901895609143
:100510000501709106018091070190910801E7E0C3
:10052000660F771F881F991FEA95D1F72DE730E0F6
:1005300040E050E0CFD3CA01B9010895AF92BF9215
:10054000CF92DF92EF92FF920F931F935B016C01AA
:10055000DEDF7B018C01DBDF6E197F09800B910BE5
:100560006A157B058C059D05B0F31F910F91FF90D7
:10057000EF90DF90CF90BF90AF900895019749F032
:10058000880F991F880F991F0297F8940197F1F728
:1005900078940895CFE5D4E0DEBFCDBF7894109273
:1005A000050110920601109207011092080183B70D
:1005B000826083BF83B7816083BF89B7816089BF51
:1005C0008EB582608EBD8EB581608EBD8FB5816027
:1005D0008FBD85B5846085BD85B5806485BD3F9838
:1005E0003E9A329A319A309A379A1AB8D3D1E1D1D9
:1005F000FECFCF93DF93880F991F880F991FA0918B
:100600009800B0919900A80FB91FED91FC91119736
:10061000309731F1EE0FFF1FED014A815B81672BAF
:1006200081F4EA51FF4F0190F081E02D20A181E09B
:1006300090E002C0880F991F4A95E2F78095282321
:100640000EC0EA51FF4F0190F081E02D20A181E022
:1006500090E002C0880F991F4A95E2F7282B20A34B
:10066000DF91CF910895CF93DF939C01880F991F5D
:10067000880F991FA0919800B0919900A80FB91FF9
:100680004D915C9111974115510509F444C0220F19
:10069000331FE0917A00F0917B00E20FF31F01908D
:1006A000F081E02DE230F10519F48FB58F7705C0A8
:1006B000E330F10521F48FB58F7D8FBD05C03497F0
:1006C00019F485B58F7D85BDFA01EE0FFF1FED0191
:1006D0004A815B81672B81F4E452FF4F0190F081E6
:1006E000E02D20A181E090E002C0880F991F4A957B
:1006F000E2F7809528230EC0E452FF4F0190F0816D
:10070000E02D20A181E090E002C0880F991F4A955A
:10071000E2F7282B20A3DF91CF9108959F92AF920B
:10072000BF92CF92DF92EF92FF920F931F93CF93DE
:10073000DF936C017B015A01922EC0E0D0E007E00C
:1007400010E0692D7727A114B10439F40C2E02C0F2
:10075000759567950A94E2F706C0002E02C075955C
:1007600067950A94E2F761707070C6017CDF61E002
:1007700070E0C70178DF60E070E0C70174DF2196A8
:1007800001501040C830D105E1F6DF91CF911F91A3
:100790000F91FF90EF90DF90CF90BF90AF909F9020
:1007A00008950F931F93CF93DF93EC018B0161E0CA
:1007B00070E01FDFCE01880F991FE0917A00F09161
:1007C0007B00E80FF91F0190F081E02DE230F10588
:1007D00031F48FB580688FBD1BBD0ABD1AC0E330F0
:1007E000F10531F48FB580628FBD19BD08BD11C010
:1007F000349729F485B5806285BD03BD0AC00038F1
:1008000011051CF460E070E002C061E070E0CE0110
:100810002ADFDF91CF911F910F910895CF93DF933E
:100820009C01880F991F880F991FC0919800D09143
:100830009900C80FD91FA881B981109719F480E0D9
:1008400090E02DC0220F331FE0917A00F0917B00E1
:10085000E20FF31F0190F081E02DE230F10519F471
:100860008FB58F7705C0E330F10521F48FB58F7D0B
:100870008FBD05C0349719F485B58F7D85BDAA0F4E
:10088000BB1FAE52BF4FED91FC9180A199270A800A
:1008900002C0959587950A94E2F781709070DF9178
:1008A000CF910895CF93DF93880F991F880F991FD9
:1008B000A0919800B0919900A80FB91FED91FC91FB
:1008C0001197EE0FFF1FEE52FF4F0190F081E02DC8
:1008D000ED018A819B81A1E0B0E0082E02C0AA0F41
:1008E000BB1F0A94E2F720E030E0672B11F021E013
:1008F00030E0B90102C0660F771F8A95E2F7EF0179
:10090000A09680A199278A239B2386179707C9F76A
:1009100020E030E040E050E004C02F5F3F4F4F4FF9
:100920005F4F888199278A239B2386179707A9F30E
:10093000CA01B90124E130E040E050E099D127E15B
:1009400030E040E050E0C6D1CA01B901DF91CF915B
:10095000089527B1207F880F991F880F991FE09174
:100960006000F0916100E80FF91F82818F70282BE1
:1009700027B961E070E080E090E0E0DD369A3699DA
:10098000FECF24B185B19927982F88273327822B52
:10099000932B089561E070E08091F0009091F10058
:1009A00028DE40E855E260E070E084E091E02AD083
:1009B000089584E091E02DD090930301809302018B
:1009C0002FEF8F3F9207D9F081369105C1F462EF86
:1009D00070E084E091E024D061E070E08091F0006C
:1009E0009091F10040DE68EC70E080E090E0A6DDE0
:1009F00060E070E08091F0009091F10034DE0895A5
:100A000008950895CB01BA01F3DB089522DC9927FC
:100A100008952DDC089549DC0895862F8BDC089518
:100A2000CB018DDC0895862F85DC08950F931F93ED
:100A30008C016DE0F2DF6AE0C801EFDF1F910F91DA
:100A400008950F931F938C01E8DFC801EFDF1F911A
:100A50000F9108950F931F938C01E2DFC801E6DF29
:100A60001F910F9108950F931F938C01DCDFC80134
:100A7000DDDF1F910F910895CB01BA013327442781
:100A8000552769DC08952AE0F7DF08950F931F9337
:100A90008C01F9DFC801CADF1F910F910895AB01E6
:100AA00066277727F0DF0895EF92FF920F931F9349
:100AB000CF93DF93EC017A018B0177FF0AC06DE2DF
:100AC000ACDF10950095F094E094E11CF11C011D41
:100AD000111D2AE0B801A701CE01CEDFDF91CF9131
:100AE0001F910F91FF90EF9008950F931F938C012A
:100AF000DBDFC8019BDF1F910F91089521153105A0
:100B000019F4642F8ADF08952A30310511F4CCDFFF
:100B10000895B2DF08950F931F938C01EFDFC80192
:100B200085DF1F910F910895AB01662757FD6095F2
:100B3000762FBADF08950F931F938C01F5DFC8015C
:100B400075DF1F910F91089508950895009709F09A
:100B500084D00895EF92FF920F931F937B018C0135
:100B6000611571058105910529F460E070E080E070
:100B700090E00AC06ED0AA2797FDA095BA2FBC01BD
:100B8000CD01A8019701C8D01F910F91FF90EF9060
:100B90000895EF92FF920F931F937B018C016217D0
:100BA0007307840795075CF4261B370B480B590B1A
:100BB000CA01B901CFDFE60EF71E081F191FC801D1
:100BC000B7011F910F91FF90EF900895A0E0B0E062
:100BD000EBEEF5E0DEC0EC01E880F9800A811B81D4
:100BE000C801B7012DE133EF41E050E073D027EAAF
:100BF00031E440E050E03CD05B016C01C801B7013A
:100C00002DE133EF41E050E065D0CA01B90124E1A4
:100C10003BE040E050E02CD0A61AB70AC80AD90A37
:100C20001A141B041C041D0444F08FEF9FEFAFEF58
:100C3000BFE7A80EB91ECA1EDB1EA882B982CA82EF
:100C4000DB82C5019F77EAE0CDB7DEB7BEC0BEDF6D
:100C5000089586EF90E0BADF0895AA27BB27809316
:100C6000F6009093F700A093F800B093F900089570
:100C7000629FD001739FF001829FE00DF11D649F80
:100C8000E00DF11D929FF00D839FF00D749FF00D0C
:100C9000659FF00D9927729FB00DE11DF91F639FAD
:100CA000B00DE11DF91FBD01CF011124089597FB7F
:100CB000092E07260AD077FD04D049D006D000209F
:100CC0001AF4709561957F4F0895F6F79095819588
:100CD0009F4F0895A1E21A2EAA1BBB1BFD010DC058
:100CE000AA1FBB1FEE1FFF1FA217B307E407F507DC
:100CF00020F0A21BB30BE40BF50B661F771F881FB8
:100D0000991F1A9469F760957095809590959B014D
:100D1000AC01BD01CF01089597FB092E05260ED029
:100D200057FD04D0D7DF0AD0001C38F45095409509
:100D3000309521953F4F4F4F5F4F0895F6F79095AF
:100D40008095709561957F4F8F4F9F4F0895AA1B97
:100D5000BB1B51E107C0AA1FBB1FA617B70710F0A6
:100D6000A61BB70B881F991F5A95A9F780959095D8
:100D7000BC01CD010895EE0FFF1F0590F491E02D09
:100D800009942F923F924F925F926F927F928F922F
:100D90009F92AF92BF92CF92DF92EF92FF920F930A
:100DA0001F93CF93DF93CDB7DEB7CA1BDB0B0FB614
:100DB000F894DEBF0FBECDBF09942A8839884888D1
:100DC0005F846E847D848C849B84AA84B984C88467
:100DD000DF80EE80FD800C811B81AA81B981CE0F5E
:100DE000D11D0FB6F894DEBF0FBECDBFED01089543
:100DF0006200030000000300010003000200030082
:100E0000030003000400030005007C00FFFFFFFF58
:100E1000FFFFFFFFFFFFFFFFFFFFFFFFFFFF0200DE
:100E200003000400FFFFFFFF9A000400000004001D
:100E30000100040002000400030004000400040098
:100E40000500040006000400070002000000020084
:100E50000100020002000200030002000400020080
:100E60000500FFFFFFFF160013001000FFFFFFFF4C
:100E7000180015001200FFFFFFFF170014001100FB
:0A0E80000D00414243000100000094
:00000001FF
